:10000000B2018E2AA501A400B3172730A300103037
:1000100015200330A300E8301520A301643015201B
:10002000A3010A30152024082028A2002508A100D9
:100030002408A0004C222008031DB313B31B0800A2
:10004000303E23280408A20083168612831209304A
:10005000A30003103220A20CA30B2A280314322081
:100060000314892A031837280000861239288616B7
:1000700039280030A1006230F829B216B21EB2123F
:10008000B2194628B2157F2003186D280830A30046
:100090009320A20DA30B4828B21E78209D20992002
:1000A000B21A6D20722022080310892AB216B21EDD
:1000B000B21232196028FE39B30032150310892AB2
:1000C000321A6828A60032167F2003186D282608E9
:1000D000862003186D28B21E892A78209D203211AF
:1000E0003212B211360884003408841780047E2846
:1000F00036088400340980058417800508007220C2
:100100009D20782099203308B2190138A2000830C8
:10011000A300A20D03187220031C78209D209920B3
:10012000A30B892872209D2036088400340800051E
:10013000FF3E3708840035097B28370884003508DE
:100140007528083033190130A300A2013608840055
:100150003408C221340880048922892284130005CE
:10016000FF3E331DA20C3319A20D3230F721A30B31
:10017000A82822080314892AA20008303319013064
:10018000A300A20C360884003408C22134080318E6
:1001900080043730F72134088004A30BC1280314EE
:1001A000892AB31C892AD728B300331C892A360828
:1001B00084003408C2210130A100E030F821340865
:1001C00080040130A100E030F829B40084178004D5
:1001D0008413A201201CA20007210319892A0721E8
:1001E0000319892A0721892AB400C521200821047E
:1001F0000319892A7E2284133408800664000029AA
:100200000129A00A0319A10FFE288006892A3408B3
:10021000A2060130A000A101000834052206031D3A
:100220000800A00A0319A10F0C2908003708A00034
:100230003508A1000130A200A30164003E21031C87
:100240003129A20B1D29FF30A30703181D29A00780
:10025000031CA107031C08006430A2000030A300A7
:100260001D296F210830A30070213E21A20C3829DE
:10027000A30B3429702103142208080036088400D7
:100280003408841780048413000533193406FF3EB4
:100290000800A600360884000930A7000310552185
:1002A000A60CA70B4F29031455298413B31D6429E9
:1002B00000083404331D3406800084170008340419
:1002C000031C34068000702900083404031C340623
:1002D00033193406800084173409800570293317D8
:1002E00001308A00330D0639A0008221A1000130BF
:1002F0008A00200A8221331FF8293313A00002301C
:100300001922F829863E03188A0A820001348B34A8
:1003100003342B34003452340C34EF34A400290855
:100320000319892A8422A000251883172408840031
:10033000200880008313A40AA9038F29B313290876
:100340000319B3170430A800250EAB212508AB21F3
:10035000240EAB2124080F39F63E0318073E0A3E4F
:10036000B129A000A8030319B31329080319BB2955
:100370002802031808002008031DB313B31B08004C
:10038000303E842AFF3A8005C629FF3A841780054B
:10039000892A83178001840AFF3E031DCA29892AFE
:1003A000031783168C010C1483120C0803178D0A93
:1003B000892A030103178C0083168C010C15553014
:1003C0008D00AA308D008C148C18E4290C11831236
:1003D0008D0A892AA301A200FF30A207031CA307EC
:1003E000031C892A0330A100E330F821EC29A10184
:1003F000F43EA000A109FE30031C012AA007031847
:10040000FE29A0076400A10FFE2900002018082A79
:1004100020180A2A08002E220E2A28220319142A3C
:100420002308A1002208A000200808000310A10C46
:10043000A00CFF3E0318162A2008892AA2000230C9
:10044000312AA101A301A2000330312AA101A30195
:10045000A2000130312AA2000630312AA200043065
:10046000312AA80023082102031D382A220820026D
:10047000043003180130031902302805031DFF3032
:10048000892A0038031DFF300405031DFF30892A27
:100490000404031DFF30892AA501A4011030A60021
:1004A000210DA40DA50D2208A4022308031C230F6F
:1004B000A5020318622A2208A40723080318230FA1
:1004C000A5070310A00DA10DA60B502A2008892A0C
:1004D0001030A800A101A001A70CA60C031C762ACD
:1004E0002208A00723080318230FA107A10CA00CC2
:1004F000A50CA40CA80B6C2A2408892AA009A10920
:10050000A00A0319A10A0800840031088A003008F3
:10051000820083130313831264000800C0309F001D
:10052000831675308F008312031787018801031328
:10053000393090008316FF30850086019F30870098
:1005400003170F30880089018312031341309F0085
:10055000831680309F0083122030840060308A012F
:10056000CA21A030840050308A01CA211030840092
:1005700060308A01C9219030840060308A01C9212D
:1005800020308600871207130317FC308D000313F9
:100590008A01D021D2000317FD308D0003138A0198
:1005A000D021D3000317FE308D0003138A01D02120
:1005B000E2000317FF308D0003138A01D021E3000E
:1005C0000317FA308D0003138A01D021C8000317E6
:1005D000FB308D0003138A01D021C9000317F830C6
:1005E0008D0003138A01D021DA000317F9308D0042
:1005F00003138A01D021DB000317F4308D000313AD
:1006000052088A01DA210317F5308D0003135308CD
:100610008A01DA210317F6308D0003135A088A0184
:10062000DA210317F7308D0003135B088A01DA2102
:1006300006148316061083120330A300E8308A01E3
:10064000EB210610831606101B3083128A0123202B
:1006500046308A0123201B308A0123202E308A0154
:1006600023201B308A01232043308A01232042307B
:100670008A0123204D308A01232053308A01232010
:1006800020308A0123204D308A01232061308A01E5
:10069000232073308A01232074308A01232065309F
:1006A0008A01232072308A01232020308A012320EE
:1006B00056308A01232030308A0123202E308A01CF
:1006C000232030308A01232037308A012320423012
:1006D0008A01232079308A01232020308A012320B7
:1006E00050308A01232065308A01232074308A012A
:1006F000232065308A01232072308A012320203094
:100700008A01232050308A01232065308A0123206A
:1007100072308A0123206B308A01232069308A01DC
:1007200023206E308A01232073308A012320773002
:100730008A01232077308A01232077308A01232001
:100740002E308A01232031308A01232035308A015E
:10075000232030308A0123206D308A01232070301D
:100760008A01232067308A0123202E308A0123202A
:1007700063308A0123206F308A0123202E308A01C2
:10078000232075308A0123206B308A0123200A3010
:100790008A0123200D308A01232038308A0123204A
:1007A0006D308A01232068308A0123207A308A0143
:1007B000232020308A01232028308A012320013081
:1007C0008A01022029308A01232020308A01232037
:1007D00043308A01232065308A0123206C308A014E
:1007E00023206C308A01232073308A01232021309A
:1007F0008A0123200730A300D0308A01EB211B306F
:100800008A01232043308A012320DB30D6000B30BD
:10081000D70056088E0057088F000C100830860647
:100820008316861183128A110A12A6248A150A12C7
:100830005B218A150A120A208A150A1254238A1586
:100840000A12DF2664006908043C8A110A12031D9B
:100850002C2C8A150A1280276400013070028A113C
:100860000A12031C372CF10A8A110A12382CF101E2
:100870008A110A1644227108A00002308A0121223E
:10088000DC007008A00000308A012622DE005C082F
:1008900084005E088A014122DE00DF0064005E08F9
:1008A0005F048A110A120319582C8A150A120C25A2
:1008B000F001FA0A64007A08283C8A110A12031D22
:1008C0009A2C0317FC308D00031352088A01DA2199
:1008D0000317FD308D00031353088A01DA21031733
:1008E000FE308D00031362088A01DA210317FF30FE
:1008F0008D00031363088A01DA210317FA308D0093
:10090000031348088A01DA210317FB308D00031313
:1009100049088A01DA210317F8308D0003135A08B9
:100920008A01DA210317F9308D0003135B088A016D
:10093000DA21FA0164008A110A120C1C9A2C56085A
:100940008E0057088F000C108A010E2C0615831696
:100950000611033083128A01EA210611831606115B
:10096000013083128A01EA212830A000A10106305B
:10097000840004308A01F420FF30E600E701D4014E
:10098000D50132308A01EA2106158316061103309B
:1009900083128A01EA21061183160611013083129F
:1009A0008A01EA211430A000A1010630840004303D
:1009B0008A01F4200130E4006400023064028A11EC
:1009C0000A1203183B2DC201C3010730B600803064
:1009D000B4000630B3006430B700B5018A011621B7
:1009E0008A110A12031C3B2FC200640042086702EE
:1009F0008A110A120318002D4208E7006408F70064
:100A00006400660842028A110A1203180B2D42087C
:100A1000E6006408F800AF30C2070318C30A4208B2
:100A2000A0004308A1000130A3007C308A012B22E2
:100A30008A110A12031D202D0130F0006408F6000F
:100A40004208A0004308A100A301DC308A01232250
:100A50008A110A12031D302D0230F0006408F600DE
:100A60004208D40743080318013ED507E40A8A1157
:100A70000A12031DDC2C061583160611033083129F
:100A80008A01EA21061183160611013083128A01B8
:100A9000EA213C30A000A1010630840004308A0124
:100AA000F42064007408013C8A110A12031D802D91
:100AB0005408A0005508A1004F08A3004E088A0161
:100AC00023228A110A12031D7C2D5408CE025508D8
:100AD000031C013ECF024E08A0004F08A100A30155
:100AE00032308A012B228A110A12031D792D063019
:100AF000F0008A110A12802D5408CE005508CF004C
:100B00005408A0005508A1006430A200A3018A0186
:100B10004C22E4002108E5005408A0005508A1007B
:100B20006430A200A3018A014C222408DC002508BD
:100B3000DD005C08A0005D08A1000A30A200A3014E
:100B40008A014C22E8002108E9006408FF001B30FC
:100B50008A01232053308A01232000308A01232078
:100B600000308A01232056308A0123206F308A0109
:100B700023206C308A01232020308A01232065083D
:100B8000A50064088A0103202E308A012320690809
:100B9000A50068088A01032020308A0123205630EE
:100BA0008A01232020308A012320AF306707E40028
:100BB000E501E50D6408A0006508A1000130A3006F
:100BC0006D308A012B228A110A12031DF22D861420
:100BD00083168610831207178316071383128A1150
:100BE0000A12F62D07138316071383126408A00058
:100BF0006508A1006430A200A3018A014C22E8002C
:100C00002108E9006408A0006508A1006430A20082
:100C1000A3018A014C222408EA002508EB0077088A
:100C2000E4001B308A01232053308A012320003046
:100C30008A01232001308A01232048308A012320A1
:100C400069308A01232056308A01232020308A010E
:100C500023205B308A01232064000A3064028A1159
:100C60000A120318362E30308A0123206A08A000A9
:100C70006B08A100A3010A308A0123228A110A12FB
:100C8000031D672E64088A0102205D308A0123203B
:100C900020308A0123206908A50068088A01032002
:100CA0002E308A01232030308A0123206B08A500D2
:100CB0006A088A01032020308A01232056308A01E5
:100CC000232020308A0123208A110A12862E6408EC
:100CD0008A0102205D308A01232020308A012320EE
:100CE0006908A50068088A0103202E308A012320A4
:100CF0006B08A5006A088A01032020308A0123209E
:100D000056308A01232020308A012320AF30660725
:100D1000E400E501E50D6408A0006508A100A30159
:100D2000E6308A0123228A110A12031DA22E06161A
:100D300083160612831287168316871283128A116E
:100D40000A12AA2E0612831606128312871283161F
:100D5000871283126408A0006508A1006430A20015
:100D6000A3018A014C22E8002108E9006408A000E0
:100D70006508A1006430A200A3018A014C22240866
:100D8000EA002508EB007808E4001B308A012320E4
:100D900053308A01232000308A01232002308A0147
:100DA00023204C308A0123206F308A0123205630C3
:100DB0008A01232020308A0123205B308A012320EE
:100DC00064000A3064028A110A120318EA2E3030D5
:100DD0008A0123206A08A0006B08A100A3010A3041
:100DE0008A0123228A110A12031D1B2F64088A011B
:100DF00002205D308A01232020308A0123206908E7
:100E0000A50068088A0103202E308A012320303093
:100E10008A0123206B08A5006A088A01032020307C
:100E20008A01232056308A01232020308A01232082
:100E30008A110A123A2F64088A0102205D308A0161
:100E4000232020308A0123206908A50068088A0130
:100E500003202E308A0123206B08A5006A088A012E
:100E6000032020308A01232056308A01232020309D
:100E70008A01232008006408F6000330F00008000F
:100E8000E601E701E401E50149309F000130E90096
:100E900064000B3069028A110A120318682F9F142C
:100EA00064008A110A129F1C572F8A01502F1E08B6
:100EB000EB0083161E088312EA006A08E4076B0839
:100EC0000318013EE507E90A8A110A12031D482F9B
:100ED0004D309F000130E90064000B3069028A1137
:100EE0000A1203188C2F9F1464008A110A129F1C87
:100EF0007B2F8A01742F1E08ED0083161E088312B3
:100F0000EC006C08E6076D080318013EE707E90AE4
:100F10008A110A12031D6C2F6608A0006708A10041
:100F20000A30A200A3018A014C22E6002108E70052
:100F30006408A0006508A1000A30A200A3018A018C
:100F40004C22E4002108E50030306402DC0002306D
:100F5000031C013E6502DD005D0C5C0CFC003030C2
:100F60006602DC000230031C013E6702DD005D0CFE
:100F70005C0CFD007C08A00032308A012622DC00D7
:100F80007D08A00032308A012622DE005C08840041
:100F90005E088A014822DE00DF0064005E085F040C
:100FA0008A110A120319D62F0430F0001B308A016F
:100FB000232053308A01232000308A01232003306C
:100FC0008A01232054308A01232065308A0123209E
:100FD0006D308A01232020308A01232046308A0187
:100FE000232064088A01022020308A012320523005
:100FF0008A01232066088A01022020308A012320EA
:10100000F8308A01232043308A01232020308A01CE
:10101000232008001B308A01232053308A0123201B
:1010200000308A01232003308A01232054308A01B2
:10103000232065308A0123206D308A01232020304F
:101040008A0123200730B6000430B40001308A0141
:10105000D42055308A01BC2028308A01BC20D630EB
:101060008A01BC202D308A01BC2016308A01BC20A8
:1010700001308A01BC2000308A01BC2000308A0186
:10108000BC20E6308A01BC20BE308A01BC208A0127
:10109000D1208A150A12FF201B308A0123205330E9
:1010A0008A01232000308A01232003308A01232073
:1010B00054308A01232065308A0123206D308A0153
:1010C000232020308A01232066088A0123206A0811
:1010D0008A0102202E308A0123206B088A01022017
:1010E00020308A0123200730B6000430B4000130DC
:1010F0008A01D42055308A01BC2028308A01BC20C6
:10110000D6308A01BC202D308A01BC2016308A01DD
:10111000BC2001308A01BC2000308A01BC20003094
:101120008A01BC20E6308A01BC2044308A01BC2000
:101130008A01D1206A08FC000730B6000430B400F0
:1011400001308A01D42055308A01BC2028308A0120
:10115000BC20B9308A01BC2011308A01BC20163075
:101160008A01BC2001308A01BC2000308A01BC20E9
:1011700000308A01BC20A4308A01BC20BE308A0124
:10118000BC208A01D1208A150A12FF2066088A0134
:1011900023206A088A0102202E308A0123206B084E
:1011A0008A01022020308A0123200730B600043053
:1011B000B40001308A01D42055308A01BC20283087
:1011C0008A01BC20B9308A01BC2011308A01BC20C0
:1011D00016308A01BC2001308A01BC2000308A010F
:1011E000BC2000308A01BC20A4308A01BC204430DD
:1011F0008A01BC208A01D1206A08FD00080007305E
:10120000B6000430B40002308A01D4208A01A12043
:10121000E4008A01A120E5008A01D1202B30E600FC
:101220006408A0006508A100FC30A3008F308A018B
:101230002B228A150A12031D24292D30E600E50908
:10124000E409E40A0319E50A6408A6006508A70092
:101250000530A200A3018A016822DC002508DD0018
:101260005C08A0005D08A1000830A200A3018A016B
:101270004C22E4002108E5006408A0006508A100F4
:101280000A30A200A3018A014C22EA006408A000EF
:101290006508A1000A30A200A3018A014C2224089B
:1012A000EB00640033306A028A150A12031C5A29C3
:1012B0000430F0000800E601E70141309F000130F2
:1012C000E50064000B3065028A150A1203188229B2
:1012D0009F1464008A150A129F1C71298A150A122C
:1012E00069291E08C10083161E088312C000400829
:1012F000E60741080318013EE707E50A8A150A12C6
:10130000031D61296608A0006708A1000A30A20039
:10131000A3018A014C22C0002108C1004008A0009E
:101320004108A1000130A300FB308A0123228A1565
:101330000A12031DBF294008FE3CDC004108031CC3
:10134000013E013CDD000330A000A101A301633098
:101350008A010D22DE002108DF005C08A0005D0884
:10136000A1005E08A2005F08A3008A014C22C00011
:101370002108C1002B30F3008A150A12F429400815
:10138000A0004108A1000230A30000308A012B22F6
:101390008A150A12031DF02900304002DC000230D9
:1013A000031C013E4102DD000330A000A101A301A6
:1013B00063308A010D22DE002108DF005C08A000F6
:1013C0005D08A1005E08A2005F08A3008A014C220C
:1013D000C0002108C1002D30F3008A150A12F4293B
:1013E000C001C1013D30F3005408A0005508A10020
:1013F0006430A200A3018A014C22DC002108DD0038
:101400005C08A6005D08A7004008A2004108A300F0
:101410008A016822E4002508E5006408A000650848
:10142000A100E830A2000330A3008A014C22240866
:10143000DC002508DD005C08A0005D08A100643028
:10144000A200A3018A014C22E6002108E7006408FB
:10145000A0006508A100E830A2000330A3008A01C3
:101460004C22E4002108E5001B308A012320533080
:101470008A01232000308A01232004308A0123209E
:1014800041308A0123206D308A01232070308A0187
:10149000232020308A01232073088A012320410859
:1014A000A50040088A01032020308A0123204B3008
:1014B0008A01232020308A0123206508A5006408C2
:1014C0008A0103202E308A0123206708A5006608C0
:1014D0008A01032020308A0123204008A600410809
:1014E000A7006430A200A3018A016822DC0025085D
:1014F000DD005C08A0005D08A1002430A200A3016B
:101500008A014C22C0002108C100640073082B3CF2
:101510008A150A12031DB82A4008C4074108031897
:10152000013EC5074408A0004508A100A3011430EE
:101530008A012E228A150A12031DB82A0130A00042
:10154000A1013A30A30098308A010D22DC00210865
:10155000DD005C08DA075D080318013EDB07143084
:10156000C4020030031C013EC5028A150A12922AE9
:10157000640073082D3C8A150A12031DEA2A4008EC
:10158000C60741080318013EC7074608A0004708E0
:10159000A100A30114308A012E228A150A12031D0C
:1015A000EA2A0130A000A101A30101308A010B2227
:1015B000DC002108DD005C08DA025D08031C013E46
:1015C000DB021430C6020030031C013EC7028A153C
:1015D0000A12C52A5A08A0005B08A1006430A200C4
:1015E000A3018A014C22E8002108E9006808FB00F9
:1015F0005A08A0005B08A1006430A200A3018A0180
:101600004C222408E4002508E5001B308A01232031
:1016100053308A01232000308A01232005308A01BB
:10162000232053308A0123206F308A012320633026
:101630008A01232020308A0123206908A500680838
:101640008A0103202E308A0123206408A000650847
:10165000A100A3010A308A0123228A150A12031D60
:10166000452B30308A0123206508A50064088A01D3
:10167000032020308A01232025308A0123202030B6
:101680008A0123208A150A12532B6508A5006408D5
:101690008A01032020308A01232025308A0123205B
:1016A00020308A01232008000130A0000730840088
:1016B00002308A01E5202008E6002108E7006608DC
:1016C000A0006708A100A30100308A011E228A152C
:1016D0000A12031D8B2B6608A0006708A1000B30BF
:1016E000A200A3018A014C22E6002108E700E430B1
:1016F000A0001E30A1006608A2006708A3008A01AE
:101700004C22DC002108DD0001305C07E6005D08AA
:101710000318013EE7001B308A01232053308A0161
:10172000232000308A01232006308A0123204D30F7
:101730008A01232070308A01232068308A01232007
:1017400020308A0123206708A50066088A0103204B
:1017500020308A01232077308A01232068308A01D3
:1017600023202F308A0123206D308A01232020304E
:101770008A0123206F08A5006E088A01032020300B
:101780008A01232020308A0123206608A6006708EA
:10179000A7009230A200A3018A016822E600250872
:1017A000E7006608C80767080318013EC90748082C
:1017B000A0004908A100CE30A30040308A012E22AB
:1017C0008A150A12031D842CFE0A0130A000A10113
:1017D0002730A3000F308A010D22DC002108DD0034
:1017E0005C08E2075D080318013EE3076400640833
:1017F0000A3C8A150A12031D7B2CD20A0319D30A4C
:101800000317F4308D0003138A01D021E40003177D
:10181000F5308D0003138A01D021E5000317F6305F
:101820008D0003138A01D021E8000317F7308D00E3
:1018300003138A01D021E90064085202E40065081C
:10184000031C013E5302E5005A086802E6005B08EB
:10185000031C013E6902E7006608A0006708A100BA
:101860006408A2006508A3008A014C22E800210850
:10187000E9005A08A0005B08A1006808A2006908F6
:10188000A3008A014C22EA002108EB006A08CA0082
:101890006B08CB006808A6006908A7000430A20006
:1018A000A3018A016822DC002508DD005C08A6008F
:1018B0005D08A7001030A200A3018A016822DC00A5
:1018C0002508DD006430A000A1010330A300E7304B
:1018D0008A010D22DE002108DF005C08A0005D08FF
:1018E000A1005E08A2005F08A3008A014C22EE005E
:1018F0002108EF00FE014030C802CE30031C013E3B
:10190000C9028A150A12D72B1B308A0123205330B3
:101910008A01232000308A01232007308A012320F6
:101920004F308A01232064308A0123206F308A01DE
:10193000232020308A0123205308A50052088A0161
:10194000032020308A01232052308A012320653071
:101950008A0123206D308A01232020308A01232030
:101960004B08A5004A088A01032020308A01232061
:101970006208A0006308A1000A30A200A3018A0146
:101980004C22E4002108E5006208A0006308A100E1
:101990000A30A200A3018A014C222408E60025088F
:1019A000E7001B308A01232053308A0123200030B6
:1019B0008A01232008308A01232054308A01232001
:1019C00072308A01232069308A01232020308A0165
:1019D00023206508A50064088A0103202E308A01AF
:1019E00023206708A50066088A01032020308A01A9
:1019F000232043308A01232068308A012320673066
:101A00008A01232020308A01232074088A010220C1
:101A100020308A01232008001B308A0123205E30F9
:101A20008A01232064308A01EA211B308A012320A5
:101A300021308A0123201B308A01232043308A0170
:101A4000232020308A0123202A308A0123202030BD
:101A50008A01232042308A0123204D308A0123202D
:101A600053308A01232020308A01232041308A010B
:101A700023206C308A01232061308A0123207230B8
:101A80008A0123206D308A01232073308A012320AC
:101A900020308A0123202A308A01232020308A0125
:101AA00023200A308A0123200D308A0123200614C6
:101AB0008316061083128614831686108312061668
:101AC0008316061283120613831606138312F4017B
:101AD00064007008013C8A150A12031D992D4330D9
:101AE0008A01232065308A0123206C308A0123205B
:101AF0006C308A01232020308A01232076088A0155
:101B0000022020308A0123203E308A0123204130E8
:101B10008A0123204D308A01232061308A0123204D
:101B200078308A01232056308A01232020308A0110
:101B3000232064007008023C8A150A12031DCA2D76
:101B400043308A01232065308A0123206C308A01CA
:101B500023206C308A01232020308A01232076083C
:101B60008A01022020308A0123203C308A01232070
:101B700041308A0123204D308A01232069308A01B7
:101B800023206E308A01232056308A012320203002
:101B90008A01232064007008033C8A150A12031D81
:101BA000F82D43308A01232065308A0123206C30D0
:101BB0008A0123206C308A01232020308A012320CF
:101BC00076088A01022020308A01232045308A01CC
:101BD000232072308A01232072308A0123206F3043
:101BE0008A01232072308A01232021308A01232098
:101BF00064007008043C8A150A12031D2F2E503011
:101C00008A01232061308A01232063308A01232046
:101C10006B308A0123203E308A01232041308A0123
:101C2000232062308A01232073308A0123204D3023
:101C30008A01232061308A01232078308A01232001
:101C400054308A01232065308A0123206D308A01B7
:101C5000232070308A01232020308A012320640051
:101C60007008053C8A150A12031D662E20308A0171
:101C7000232020308A01232041308A0123206C3028
:101C80008A01232061308A01232072308A012320B7
:101C90006D308A01232020308A01232054308A01AC
:101CA000232065308A01232073308A012320743079
:101CB0008A01232021308A01232020308A01232019
:101CC00020308A01232020308A01232064007008FC
:101CD000063C8A150A12031DCD2E20308A012320CE
:101CE00020308A01232043308A01232068308A0172
:101CF000232061308A01232072308A01232067303B
:101D00008A01232065308A01232020308A01232084
:101D100045308A0123206E308A01232064308A01F5
:101D2000232021308A01232020308A0123202030E3
:101D30008A01232020308A01232020308A01232099
:101D400056308A0123206F308A0123206C308A01AB
:101D5000232074308A01232061308A0123206730D8
:101D60008A01232065308A01232020308A01232024
:101D700044308A01232072308A0123206F308A0187
:101D8000232070308A01232020308A012320203034
:101D90008A01232020308A012320F001F10107303D
:101DA000A300D0308A01EB210610831606101B30E9
:101DB00083128A0123205F308A01232008004530E6
:101DC0009F000A308A01EA219F1464008A150A12D2
:101DD0009F1CED2E8A150A12E52E1E08EB008316B5
:101DE0001E088312EA006A08A0006B08A1000430F4
:101DF000A200A3018A014C22EA002108EB00063070
:101E0000EA070318EB0A6A08A0006B08A1002A3051
:101E1000A200A3018A014C22EA002108EB00013054
:101E2000EA020030031C013EEB026A08E9000800E8
:101E3000E201E3010317FE308D00031362088A01FB
:101E4000DA210317FF308D00031363088A01DA21BA
:101E50008A110A16E328D201D3010317FC308D0042
:101E6000031352088A01DA210317FD308D00031392
:101E700053088A01DA218A110A16E3280530F00096
:101E800008001030DA002730DB000317F8308D002F
:101E900003135A088A01DA210317F9308D0003135E
:101EA0005B088A01DA218A110A16E32864000130EE
:101EB00070028A150A12031C5E2F08006400740861
:101EC000003C8A150A12031D782F0130F400861099
:101ED00083168610831206128316061283120617C3
:101EE000831606138312CE01CF018A150A127D2FA5
:101EF000F40106138316061383128A110A16E328C7
:101F00001B308A0123205E308A01232064308A013D
:101F1000EA211B308A01232043308A0123202A3002
:101F20008A01232020308A01232020308A012320A7
:101F300053308A01232075308A01232062308A01C0
:101F4000232020308A0123204D308A012320653050
:101F50008A0123206E308A01232075308A012320D4
:101F600020308A01232031308A01232020308A0149
:101F7000232020308A0123202A308A0123200A309E
:101F80008A0123200D308A01232053308A01232027
:101F900074308A01232061308A01232072308A0143
:101FA000232074308A01232020308A0123204330EB
:101FB0008A01232068308A01232061308A0123208E
:101FC00072308A01232067308A01232065308A011C
:101FD000232020308A0123203D308A012320203015
:101FE0008A01232055308A01232052308A01232080
:101FF00065308A01232073308A01232065308A01ED
:10200000232074308A01232020308A01232053307A
:102010008A0123206F308A01232063308A01232024
:1020200020308A01232020308A01232020308A0199
:10203000232020308A0123203D308A0123202030B4
:102040008A0123204C308A01232052308A01232028
:1020500065308A01232073308A01232065308A018C
:10206000232074308A01232020308A012320543019
:102070008A01232072308A01232069308A012320BB
:1020800070308A01232020308A01232020308A01E9
:10209000232020308A0123203D308A012320203054
:1020A0008A01232044308A01232052308A012320D0
:1020B00065308A01232073308A01232065308A012C
:1020C000232074308A01232020308A0123204F30BE
:1020D0008A01232064308A0123206F308A01232063
:1020E00020308A01232020308A01232020308A01D9
:1020F000232020308A0123203D308A0123202030F4
:102100008A01232052308A01232053308A01232060
:1021100075308A01232062308A01232020308A0111
:1021200023204D308A01232065308A0123206E3020
:102130008A01232075308A01232020308A01232040
:1021400032308A01232020308A01232020308A0166
:10215000232020308A0123203D308A012320203093
:102160008A01232043308A0123200730A300D03086
:102170008A01EB218A150A12DF2664006908003CF7
:102180008A150A120319562F64006908013C8A1542
:102190000A120319412F64006908023C8A150A12C9
:1021A0000319182F64006908033C8A150A120319E1
:1021B0002B2F64006908043C8A110A160319EA28C7
:1021C0008A110A16BA281B308A0123205F308A013F
:1021D000232008001B308A01232043308A0123205A
:1021E0002A308A01232020308A01232020308A01CE
:1021F000232053308A01232075308A012320623046
:102200008A01232020308A0123204D308A01232097
:1022100065308A0123206E308A01232075308A01BF
:10222000232020308A01232032308A0123202030CD
:102230008A01232020308A0123202A308A0123208A
:102240000A308A0123200D308A01232043308A017D
:10225000232065308A0123206C308A0123206C30D2
:102260008A01232020308A01232056308A0123202E
:102270006F308A0123206C308A01232074308A0158
:10228000232061308A01232067308A0123206530B2
:102290008A01232020308A0123203D308A01232017
:1022A00020308A01232055308A01232053308A01AF
:1022B00023206C308A01232061308A01232076306C
:1022C0008A01232065308A01232020308A012320BF
:1022D00055308A01232070308A01232064308A011E
:1022E000232061308A01232074308A012320653045
:1022F0008A01232020308A0123203D308A012320B7
:1023000020308A0123204C308A01232054308A0156
:10231000232078308A01232020308A012320423074
:102320008A0123204D308A01232053308A01232043
:1023300020308A01232044308A01232061308A0121
:10234000232074308A01232061308A012320203029
:102350008A01232020308A0123203D308A01232056
:1023600020308A01232044308A01232054308A01FE
:10237000232065308A0123206D308A0123207030AC
:102380008A01232020308A01232052308A01232011
:102390006F308A0123206D308A01232020308A018A
:1023A000232020308A01232020308A01232020305E
:1023B0008A01232020308A0123203D308A012320F6
:1023C00020308A01232052308A01232045308A019F
:1023D000232078308A01232069308A012320743039
:1023E0008A01232020308A01232020308A012320E3
:1023F00020308A01232020308A01232020308A01C6
:10240000232020308A01232020308A0123202030FD
:102410008A01232020308A0123203D308A01232095
:1024200020308A01232043308A0123200730A30073
:10243000D0308A01EB218A150A12DF266400690870
:10244000003C8A110A160319672B64006908013CD5
:102450008A110A160319A02C64006908023C8A112B
:102460000A160319A32A64006908033C8A150A1690
:102470000319282864006908043C8A110A16031904
:10248000E3288A110A161B2A0730B6001030B40060
:102490000730B7000830B500A0308A015820510835
:1024A0008A01582050088A01582070088A01562055
:1024B000D00A0319D10A0630B6008030B4000430C7
:1024C000B30055308A01492155308A0149215530E0
:1024D0008A01492155308A01492155308A01492113
:1024E0000A308A01EA210630B6008030B400043098
:1024F000B30062308A0149216D308A01492173306D
:102500008A01492100308A01492170088A01492144
:1025100076088A0149210730B6001030B400073030
:10252000B7000830B500A0308A01582051088A0150
:10253000582050088A01582076088A015620D00A6F
:102540000319D10A08001B308A01232043308A0175
:10255000232054308A01232078308A0123206430DC
:102560008A01232020308A0123205108A500500829
:102570008A01032020308A01232042308A0123204F
:1025800079308A01232074308A01232065308A0142
:10259000232073308A0123200A308A0123200A3045
:1025A0008A0123200D308A01232042308A01232012
:1025B00065308A01232020308A01232050308A018F
:1025C000232061308A01232074308A01232069305E
:1025D0008A01232065308A0123206E308A0123205E
:1025E00074308A01232021308A0123200630B6006E
:1025F0008030B4000430B30055308A014921553091
:102600008A01492155308A01492155308A014921E1
:1026100055308A01492105308A01EA210630B60089
:102620008030B4000430B30062308A0149216D303B
:102630008A01492173308A01492101308A014921E7
:1026400005308A01EA21E401E5016408A00065087B
:10265000A1005108A30050088A0128228A110A16F5
:10266000031D5B2B0730B6001030B4000730B700F5
:102670000830B500A0308A01582051088A0158203E
:1026800050088A0158208A013D20E6000630B60035
:102690008030B4000430B30066088A014921083054
:1026A0008606831686118312E40A0319E50A8A1145
:1026B0000A16031D252B0630B6008030B400043006
:1026C000B300FF308A0149218A110A169E2F1B3060
:1026D0008A01232043308A0123200130E5000615BA
:1026E00083160611033083128A01EA21061183162C
:1026F0000611013083128A01EA211430A000A101E1
:102700000630840004308A01F4200130E4006400C3
:10271000023064028A110A160318AC2BC201C301ED
:102720000730B6008030B4000630B3006430B70024
:10273000B5018A0116218A110A12031C3B2FC2001F
:102740006400640865028A110A160319AC2BE40AB6
:102750008A110A16031D872BAF30C2070318C30A5C
:102760004208A0004308A1006430A200A3018A012E
:102770004C22E6002108E7004208A0004308A1001F
:102780006430A200A3018A014C222408E800250835
:10279000E9006808A0006908A100A3010A308A01C5
:1027A00023228A110A16031D0C2C43308A01232090
:1027B00065308A0123206C308A0123206C308A0125
:1027C000232020308A01232065088A01022020303E
:1027D0008A01232020308A0123206708A50066088B
:1027E0008A0103202E308A01232030308A012320E1
:1027F0006908A50068088A01032056308A01232051
:1028000020308A0123200A308A0123200D308A01DA
:1028100023208A110A163D2C43308A01232065307B
:102820008A0123206C308A0123206C308A01232006
:1028300020308A01232065088A01022020308A0185
:10284000232020308A0123206708A50066088A011A
:1028500003202E308A0123206908A50068088A0118
:10286000032056308A01232020308A0123200A3099
:102870008A0123200D308A0123208A150A12DF26BF
:1028800064006908023C8A110A16031D3D2CE50A02
:102890006400013065028A110A16031C6F2B013097
:1028A000A300F4308A01EB210A308A0123200D3085
:1028B0008A01232041308A0123206E308A0123209F
:1028C00079308A01232020308A0123204B308A016D
:1028D000232065308A01232079308A01232020308B
:1028E0008A01232054308A0123206F308A0123205B
:1028F00020308A01232045308A01232078308A0144
:10290000232069308A01232074308A01232021305A
:102910008A0123200330A300E8308A01EB218A15C5
:102920000A12DF2664006908053C8A110A16031999
:102930008F2C1B308A0123205F308A01232008005E
:102940000930E8001B308A01232043308A0123200C
:102950002A308A01232020308A01232053308A0123
:1029600023206C308A01232061308A0123207630B5
:102970008A01232065308A01232020308A01232008
:1029800055308A01232070308A01232064308A0167
:10299000232061308A01232074308A01232065308E
:1029A0008A01232020308A0123202A308A01232013
:1029B00020308A01232055308A01232073308A0178
:1029C000232065308A01232020308A0123205530BE
:1029D0008A01232070308A0123202F308A0123208E
:1029E00044308A0123206F308A01232077308A0106
:1029F00023206E308A01232020308A012320743066
:102A00008A0123206F308A01232020308A0123206D
:102A100020308A01232053308A01232065308A0127
:102A200023206C308A01232065308A012320633003
:102A30008A01232074308A01232020308A01232038
:102A400043308A0123206F308A0123206D308A01B0
:102A500023206D308A01232061308A0123206E30CB
:102A60008A01232064308A01232020308A01232018
:102A70000A308A0123200D308A01232020308A0168
:102A8000232043308A01232065308A0123206E30C1
:102A90008A01232074308A01232072308A01232086
:102AA00065308A01232020308A01232050308A019A
:102AB000232075308A01232073308A012320683057
:102AC0008A01232020308A01232074308A012320A8
:102AD0006F308A01232020308A01232020308A0190
:102AE000232053308A01232065308A0123206E3051
:102AF0008A01232064308A01232020308A01232088
:102B000043308A0123206F308A0123206D308A01EF
:102B100023206D308A01232061308A0123206E300A
:102B20008A01232064308A01232021308A01232056
:102B300021308A0123200330A300E8308A01EB21F1
:102B40008A150A12DF261B308A01232053308A019E
:102B5000232000308A01232007308A0123202030DF
:102B60008A01232043308A0123206F308A012320E9
:102B70006D308A0123206D308A01232061308A0163
:102B800023206E308A01232064308A0123202030E4
:102B90008A01232068088A01022020308A0123202C
:102BA00021308A01232020308A0123200130A30014
:102BB000F4308A01EB2164006908053C8A110A1689
:102BC0000319A02D64006908003C8A110A16031D30
:102BD000EA2DE80A64006908023C8A110A16031DFE
:102BE000F22DE80364006908043C8A110A16031DEB
:102BF000A02D0A308A0123200A308A0123200D30BB
:102C00008A01232043308A0123206F308A01232048
:102C10006E308A01232066308A01232069308A01C0
:102C2000232072308A0123206D308A012320203036
:102C30008A01232020308A01232028308A01232082
:102C400059308A0123202F308A0123204E308A01F7
:102C5000232029308A01232020308A0123203F307D
:102C60008A01232020308A01232055308A01232025
:102C700070308A0123203D308A01232059308A0197
:102C8000232065308A01232073308A0123202030DD
:102C90008A01232044308A0123206F308A012320B7
:102CA00077308A0123206E308A0123203D308A014B
:102CB00023204E308A0123206F308A0123200330E5
:102CC000A300E8308A01EB218A150A12DF2664008E
:102CD0006908003C8A110A160319782E64006908F5
:102CE000023C8A110A1603199E2F8A110A16642EB5
:102CF0001B308A01232043308A01232043308A017C
:102D000023206F308A0123206D308A0123206D300B
:102D10008A01232061308A0123206E308A0123201A
:102D200064308A01232020308A01232068088A0128
:102D3000022020308A01232053308A01232065306D
:102D40008A0123206E308A01232074308A012320D7
:102D50006808A600A7011430A200A3018A01682216
:102D6000EA002508EB0006158316061103308312CE
:102D70008A01EA21061183160611013083128A01A5
:102D8000EA216A08A0006B08A10006308400043024
:102D90008A01F4200130E4006400023064028A11E8
:102DA0000A160318662F0730B6008030B4000630CC
:102DB000B300E830B7000330B5008A0116218A114C
:102DC0000A16031CE22FE900640068080C3C8A1113
:102DD0000A16031D1A2F0A308A0123200D308A019A
:102DE000232053308A0123206C308A012320613054
:102DF0008A01232076308A01232065308A0123202E
:102E000020308A01232064088A01022020308A01B0
:102E1000232056308A01232069088A0102202030AD
:102E20008A0123200130A300F4308A01EB218A11AA
:102E30000A16612F6400680869028A110A160319CC
:102E4000612F0A308A0123200D308A01232053305C
:102E50008A0123206C308A01232061308A012320DB
:102E600076308A01232065308A01232020308A01B0
:102E7000232064088A01022020308A012320453063
:102E80008A01232072308A01232072308A01232094
:102E90006F308A01232072308A01232021308A0179
:102EA000232006148316061083120B30A300B830BB
:102EB0008A01EB2106108316061083128A110A1666
:102EC0009E2FE40A8A110A16031DCC2E0A308A01AD
:102ED00023200D308A01232041308A0123206330D2
:102EE0008A0123206B308A0123206E308A0123203F
:102EF0006F308A01232077308A0123206C308A01C9
:102F0000232065308A01232064308A012320673022
:102F10008A01232065308A01232064308A0123201E
:102F200020308A0123204F308A0123204B308A0130
:102F300023200330A300E8308A01EB210A308A0104
:102F400023200D308A01232041308A0123206E3056
:102F50008A01232079308A01232020308A0123200E
:102F60004B308A01232065308A01232079308A0181
:102F7000232020308A01232054308A0123206F30FF
:102F80008A01232020308A01232045308A01232012
:102F900078308A01232069308A01232074308A0125
:102FA00023208A150A12DF2664006908053C8A116D
:102FB0000A160319D12F1B308A0123205F308A01A2
:102FC000232008000A308A0123200D308A012320A3
:102FD0002A308A01232020308A01232043308A01AD
:102FE00023206F308A0123206D308A0123206D3029
:102FF0008A01232073308A01232020308A01232074
:1030000045308A01232072308A01232072308A01E0
:1030100023206F308A01232072308A01232021303F
:103020008A01232020308A0123202A308A0123208C
:1030300006148316061083120B30A300B8308A01E1
:10304000EB2106108316061083128A110A169E2F92
:103050000730B6000430B40001308A01D420333088
:103060008A01BC208A01D1200730B6000430B400A8
:1030700000308A01D4200830A900A130B000B1018D
:10308000A50138308A018E218A01D1201B308A01A6
:10309000232043308A01232046308A0123206130D7
:1030A0008A0123206D308A01232069308A01232080
:1030B0006C308A01232079308A01232020308A0154
:1030C00023203D308A01232020308A012320023032
:1030D000A9003808A400A5012230B000B1018A017E
:1030E0009E2168308A0123200A308A0123200A3079
:1030F0008A0123200D308A0123200230A9003908DB
:10310000A400A5012230B000B1018A019E21203027
:103110008A0123200230A9003A08A400A501223028
:10312000B000B1018A019E2120308A0123200230A3
:10313000A9003B08A400A5012230B000B1018A011A
:103140009E2168308A0123200A308A0123200D3015
:103150008A0123200230A9003C08A400A5012230E6
:10316000B000B1018A019E2120308A012320023063
:10317000A9003D08A400A5012230B000B1018A01D8
:103180009E2120308A0123200230A9003E08A4009D
:10319000A5012230B000B1018A019E2168308A0168
:1031A00023200A308A0123200A308A0123200D308F
:1031B0008A01232043308A01232052308A012320B0
:1031C00043308A01232020308A01232056308A018F
:1031D000232061308A0123206C308A012320203093
:1031E0008A0123203D308A01232020308A012320B8
:1031F0000230A9003F08A400A5012230B000B101AF
:103200008A019E2168308A0123200730A300D03034
:0A3210008A01EB218A110A169E2F95
:02400E00F42399
:00000001FF
